:03000000023EF9C4
:0C3EF90078FFE4F6D8FD75816F023F40B1
:1016B80020000A3C2E2E2E3E004950436F6E6E6568
:1016C80063745245510A004950436F6E6E656374E6
:1016D800000A49504E6F41434B210A003E432C56A5
:1016E8002C43432CC0E4E0EFF2E5F020D1E8EDEA2A
:1016F800EEEC49500A003E432C4D41432C25303234
:1017080062583A25303262583A25303262583A25C2
:10171800303262583A25303262583A2530326258AF
:101728002C4D414320E0E4F0E5F10A003E432C56FD
:1017380045522C20332E3220EEF2202573202573BB
:101748002CC2E5F0F1E8FF20495020ECEEE4F3EB81
:10175800FF0A004D617220313520323031310031BD
:10176800373A30343A3533003E432C4C442C5052EF
:101778004F473A20202020202020202020202020F1
:101788002020202020202020202020202020202051
:101798002020202020202020202020202020202041
:1017A8002020202020202020202020202020202031
:1017B80020202020202020202CC4E0F2E020EFF080
:1017C800EEF8E8E2EAE828F4E0E9EB290A003E2A24
:1017D8002C312CCEF1EDEEE2EDFBE520EFE0F0E070
:1017E800ECE5F2F0FB20F1E5F2E5E2EEE3EE20E8CD
:1017F800EDF2E5F0F4E5E9F1E00A003E412C413074
:10180800312C2562752E2562752E2562752E25626E
:10181800752C495020E0E4F0E5F120E0E4E0EFF237
:10182800E5F0E00A003E412C4130322C2562752E4D
:101838002562752E2562752E2562752C495020E08B
:10184800E4F0E5F120EEF1ED2E20F1E5F0E2E5F02F
:10185800E00A003E412C4130332C2562752E25626A
:10186800752E2562752E2562752C495020E0E4F00E
:10187800E5F120F0E5E72E20F1E5F0E2E5F0E00AF9
:10188800003E412C4130342C2562752E2562752E80
:101898002562752E2562752CCCE0F1EAE020F1E591
:1018A800F2E80A003E412C4130352C2562752E2580
:1018B80062752E2562752E2562752CD8EBFEE70A17
:1018C800003E2A2C312CC4EEEF2E20EFE0F0E0ECA5
:1018D800E5F2F0FB20F1E5F2E5E2EEE3EE20E8EDDB
:1018E800F2E5F0F4E5E9F1E00A003E422C5330312C
:1018F8002C2562752CC6E4E0F2FC20E7E0EFF0EE60
:10190800F1E020F1EEE5E4E8EDE5EDE8FF20EEF2A8
:1019180020F1E5F0E2E5F0E00A003E422C533032D7
:101928002C2562752CCEE1ECE5ED20F120F1E5F0F7
:10193800E2E5F0EEEC20E1E5E720EAE2E8F2E0EDAE
:10194800F6E8E90A003E422C5330332C2562752C08
:10195800CFE5F0E5E7E0EFF3F1EA20EFF0E820EF7C
:10196800EEF2E5F0E520F1E2FFE7E820F120F1E50D
:10197800F0E2E5F0EEEC0A003E422C5330352C251F
:1019880062752CCAE0EDE0EB20F8E8F0EEEAEEE252
:10199800E5F8E0F2E5EBFCEDEEE3EE20EEE1ECE558
:1019A800EDE00A003E532C5330362C253032625875
:1019B8002530326258253032625825303262582537
:1019C8003032625825303262582C4D414320E0E4D1
:1019D800F0E5F120F8E8F0EEEAEEE2E5F8E0F2E50D
:1019E800EBFCEDEEE3EE20EEE1ECE5EDE00A003E87
:1019F800454E440A000A44756D7058202020202066
:101A08003030203031203032203033203034203014
:101A180035203036203037203038203039203041DA
:101A280020304220304320304420304520304600CA
:101A38000A3A003A20000A000A44756D70442020D2
:101A480020202030302030312030322030332030F8
:101A580034203035203036203037203038203039A7
:101A6800203041203042203043203044203045206F
:101A7800304600457272206B6579005264206565B6
:101A880070726F6D0A005264204D454D0A00526411
:101A980020436F64650A00577269746520436F6458
:101AA800650A0044656275674950204F4E0A004434
:101AB800656275674950204F46460A00446562755D
:101AC8006755736572204F6E0A00446562756755E5
:101AD800736572204F46460A0044656275674D7308
:101AE80067204F6E0A0044656275674D7367204F23
:101AF80046460A00436F6E666967206C6F636B2108
:101B08000A00577220656570726F6D0A0020536174
:101B1800766520656570726F6D210A0045727220C6
:101B28004D414321004C6F61643E3E002A003C4118
:101B380030313D003C4130323D003C4130333D00C6
:101B48003C4130343D003C4130353D003C21003CB7
:101B58005330313D003C5330323D003C5330333D2F
:0D1B6800003C5330353D003C5330363D000D
:063CF900016C00016A00ED
:10495800C28E438910E4F58B758DB8D2ABD28E2206
:03001B00023E6939
:103E6900C0E0C083C082C0D0C28E758B00758DB88A
:103E7900201E0675A61E75A6E1056AD21AE56C60B4
:103E890002056CE56BD394014002156B056FE56F74
:103E9900540F7048D226E56F543F7012D2189066BD
:103EA9008BE0600A04F0E0D394B44002D21E90661D
:103EB90086E0600204F0906104E0600214F090660C
:103EC9008CE0D394014003E014F0301D02056DE548
:103ED9006ED394644004D21E8002056EE569D394C2
:103EE9000140021569D28ED0D0D082D083D0E03281
:10104F00C291C290D2B5C2237D027C007F071249A4
:10105F00218F27E527646060097D017F601248BCFE
:10106F00D223E4FDFC7F0B1249218F27E52730E6C1
:10107F00097D04E4FF1248E0D2237D017C007F0745
:10108F001249218F27E5277008FD7FFF1248BCD238
:10109F0023302303126000C288C2A8C2AA75890038
:1010AF001242A290633EE0B4FA06A3E064CE607BE6
:1010BF00E4F52774362527F582E43463F583E4F0ED
:1010CF000527E527B443EC90633E74FAF0A374CE82
:1010DF00F0A374CCF0906344740AF0E4A3F0A3047B
:1010EF00F0A3F090633A74FFF0A3F0A3F0E4A3F041
:1010FF00906355740AF0E4F527E5272401FFE433E4
:10110F00FE74362527F582E43463F583E0FD12483B
:10111F00980527E527C3944340DFE4F5A775A61E7E
:10112F0075A6E1907FF0F0A3F080FE906349740301
:10113F00F0A374CCF0E4906348F0123C2FC2B512C8
:10114F0029FCC21E12451FD223C225C224906576E8
:10115F007408F09062B47424F0E4A3F090633EE05E
:10116F009062B6F090633FE09062B7F0906340E01A
:10117F009062B8F0906341E09062B9F0906342E002
:10118F009062BAF0906343E09062BBF0756B01E43C
:10119F00906577F0C21FC220C221C222202318AF50
:1011AF0027FE7D031238C4E4FF123DB97E167FB8C7
:1011BF00E4FBFDFC1235D190668BE060037401F007
:1011CF00E4906104F0F56D906575F0F56E12495875
:1011DF0075A70775A61E75A6E1D2AFE4F56E9061EF
:1011EF0004E070031208AB90668CE06401701D90F0
:1011FF0080007410F09080A874FFF0A3F0A3F0A308
:10120F00F0E490668CF0D223C224C225908008E0CF
:10121F00F52730E405D21F7410F0E52730E508D22A
:10122F00219080087420F0E52730E608D2209080C6
:10123F00087440F0E56DC394034019908002E4F008
:10124F00908001F0908000F0E56D94064006E4F583
:10125F006D12451F9080A0E0700312439A9080B8E2
:10126F00E070031243209080D0E070031244C390CB
:10127F008000E07013301F101236D8906331EFF0FA
:10128F00D394004003120036908002E070069080E5
:10129F0000E06005D21D0211EAC21DE4F56D9061F8
:1012AF0004E060030211EA202312906578E0600CDD
:1012BF007E167FBA1237DCE4906578F03021121277
:1012CF0031E1906331EFF0D394004005E0FF12005D
:1012DF0032202003021460122D57906331EFF0700B
:1012EF00030211EA906375E054BF247F7003021369
:1012FF00C91470030213A1240260030214022023F5
:10130F00077E167FC11237DC20270302146090631B
:10131F004DE07006906351E06067906682E0FF9049
:10132F00634DE0B50724906683E0FE90634EE0B511
:10133F000618906684E0FE90634FE0B5060C906649
:10134F0085E0FE906350E06E6037906351E06F6010
:10135F0003021460906683E0FF906352E06F6003B6
:10136F00021460906684E0FF906353E06F600302A5
:10137F001460906685E0FF906354E06F6003021481
:10138F0060C21B9065777401F0124992756B010270
:10139F00146090668BE060037401F090667AE0FF52
:1013AF00906377E06F600302146090667AE004F058
:1013BF00E4F56B906575F0021460301B0302146046
:1013CF00906344E070030211EA906355740AF012BF
:1013DF0046B0D21BE4F56B906575F090668604F00D
:1013EF00E4906679F0A3F02023677E167FCF123743
:1013FF00DC805E90668BE060037401F0301B5290CE
:10140F006375E020E74B906377E0FF906679E0FE2D
:10141F006F600D906681E07007EE146F703380136C
:10142F00906679E004F0906331E0FFD394044003B9
:10143F001233529060007482F0A37401F0906377BE
:10144F00E0906002F07E607F007D0312400C02117D
:10145F00EA201B03021578E56B706812472DEF60C9
:10146F00237E647F75906476E02404FD12400C9017
:10147F006681E07009906355E0F56B0211EAE4F5BF
:10148F006B0211EA906686E0D3943C4036906681F9
:10149F00E0703090668604F0123A80E4906475F044
:1014AF00A37412F090667AE0906477F0A374FDF065
:1014BF0090610563A20190647963A2017F121228E3
:1014CF00EE809E1249828F27E527B40115906000A8
:1014DF007483F0E4A3F07E607F007D0212400C0263
:1014EF0011EAE527D39401401C9060007483F0A3A8
:1014FF007401F0E52724FEA3F07E607F007D0312C8
:10150F00400C0211EAE56B640160030211EA906579
:10151F0075E004F02023077E167FD91237DC906325
:10152F0055E0C394C85004E02432F0906575E0C3D1
:10153F009405400DC21BE4906577F0124992021199
:10154F00EA7C667D82906349E0FAA3E0FB7F02129A
:10155F00419D7E647F75906476E02404FD12400CFB
:10156F00906355E0F56B0211EAE56B6401600302CD
:10157F0011EA906577E014604624FE604214700310
:10158F0002166B240460030211EAE4F56D202713A1
:10159F009065777404F0906575E05401F0756B01F8
:1015AF000211EA9080027410F0E4906577F0906574
:1015BF007504F0756BFA90668274FFF00211EA9071
:1015CF006682E070030216559064757480F0906423
:1015DF00777401F0E4A3F0A304F0A37430F0A374C4
:1015EF007BF0E4F527747C2527F582E43464F583DA
:1015FF00747DF0747D2527F582E43464F583E4F07F
:10160F00E5272407906476F07C667D82906349E03D
:10161F00FAA3E0FB7F0212419D7E647F75E52724CC
:10162F0009FD12400C906681E0601B1246B0D21B80
:10163F00E4F56B906575F090668604F0E49066793A
:10164F00F0A3F00211EA302707E4906577F08006E7
:10165F009065777404F0756BFA0211EA908002744A
:10166F0010F0756B05906575E06401FFF09065777C
:10167F007401F0EF7019906351E06013FCA3E0FD6B
:10168F00A3E0FEA3E0FF9066821224920211EA907B
:10169F00634DE0FCA3E0FDA3E0FEA3E0FF906682B4
:0816AF001224920211EA80FEF0
:0116B7002210
:10003600906376E0B444047F0180027F009063758C
:10004600E0B447047E0180027E00EE5F604A906362
:100056003EE0906377F090633FE0906378F09063C2
:1000660040E0906379F0906341E090637AF09063AA
:1000760042E090637BF0906343E090637CF0906392
:10008600767452F09062AE63A2019080A863A201DA
:100096007F061228EE0208A1906331E0C39408504F
:1000A600030208AA90633EE0FF906377E06F600367
:1000B6000208AA90633FE0FF906378E06F60030256
:1000C60008AA906340E0FF906379E06F600302083E
:1000D600AA906341E0FF90637AE06F60030208AA8A
:1000E600906342E0FF90637BE06F60030208AA9092
:1000F6006343E0FF90637CE06F60030208AA9063AD
:1001060076E06444701A9080A8E0B4FF139062AE63
:1001160063A2019080A863A2017F061228EE8010D8
:100126009062B2E09080ACF09062B3E09080ADF067
:1001360090668BE060037401F090668C7464F090B6
:1001460063767452F0906375E0646D60030202ABEF
:100156007BFF7A1679E4121FFE7BFF7A1679FE90F2
:10016600633EE0F534A3E0F535A3E0F536A3E0F50C
:1001760037A3E0F538A3E0F539121FFE7534FF7595
:10018600351775365B7537FF7538177539677BFF19
:100196007A177934121FFE7BFF7A177970121FFEC9
:1001A6007BFF7A1779D6121FFE7BFF7A18790390A8
:1001B6006344E0F534A3E0F535A3E0F536A3E0F5B6
:1001C60037121FFE7BFF7A18792D90634DE0F534C8
:1001D600A3E0F535A3E0F536A3E0F537121FFE7B65
:1001E600FF7A18795B906351E0F534A3E0F535A307
:1001F600E0F536A3E0F537121FFE7BFF7A18798902
:1002060090633AE0F534A3E0F535A3E0F536A3E0D4
:10021600F537121FFE7BFF7A1879AC906336E0F54E
:1002260034A3E0F535A3E0F536A3E0F537121FFE5B
:100236007BFF7A1879C9121FFE7BFF7A1879F2A222
:1002460027E433F534121FFE7BFF7A197922906674
:1002560081E0F534121FFE7BFF7A19794D90668B8B
:10026600E0F534121FFE7BFF7A197980A219E43378
:10027600F534121FFE7BFF7A1979AC90667BE0F5A8
:1002860034A3E0F535A3E0F536A3E0F537A3E0F5B2
:1002960038A3E0F539121FFE122EDE7BFF7A19799C
:1002A600F7121FFE22906375E0644C70737E197F0F
:1002B600FDFBFDFC1235D190637DE0F528A3E0F54A
:1002C60029E4F52BE52890637FF0A3E529F07E1A53
:1002D6007F387C637D7F7B021235D1E4F52A852940
:1002E60082852883E0FF747F252AF582E43463F54E
:1002F60083EFF00529E52970020528052AE52AB4C9
:1003060010DC7E1A7F3B7C637D7F7B101235D10526
:100316002BE52BC3941040AC7E1A7F3E1237DC22AD
:10032600906375E0646C7060F52C7E1A7F40FBFD6F
:10033600FC1235D1E4F52BE490637FF0A3E52CF0B5
:100346007E1A7F387C637D7F7B021235D1E4F52AE5
:10035600A82CE6FF747F252AF582E43463F583EF43
:10036600F0052C052AE52AB410E67E1A7F3B7C634D
:100376007D7F7B101235D1052BE52BC3940840B742
:100386007E1A7F3E1237DC22906375E0644B706103
:10039600F52A7467252AF582E43463F583E0603232
:1003A6007467252AF582E43463F583E0F4602374E8
:1003B60067252AF582E43463F583E0FF747D252AF8
:1003C600F582E43463F583E0B50710052AE52AB41F
:1003D60008C09061047432F00208A190637574211C
:1003E600F03023030208A17E1A7F7B1237DC020855
:1003F600A1906375E0B4521A2023077E1A7F8312F8
:1004060037DC9063757472F07E637F757D08123FEA
:100416008522906375E0644970452023077E1A7F24
:100426008E1237DC90637DE0F528A3E0F529E4F52C
:100436002A852982852883E0FF747F252AF582E4B0
:100446003463F583EFF00529E52970020528052AAE
:10045600E52AB480DC7E637F757D8A123F85229013
:100466006375E0644370462023077E1A7F96123731
:10047600DC90637DE0F528A3E0F529E4F52A8529DB
:1004860082852883E493FF747F252AF582E434630A
:10049600F583EFF00529E52970020528052AE52AE6
:1004A600B480DB7E637F757D8A123F8522906375FB
:1004B600E0645A70532023077E1A7F9F1237DC9020
:1004C600637DE0F528A3E0F5297C637D7F7B80AF23
:1004D60029AE2812480DE4F52A852982852883E469
:1004E60093FF747F252AF582E43463F583EFF005E4
:1004F60029E52970020528052AE52AB480DB7E63F2
:100506007F757D8A123F8522906375E0644460039F
:1005160002059F90637DE0FF644470030208A1EF2B
:10052600B4310CC2237E1A7FAB1237DC0208A190CD
:10053600637DE0B4300CD2237E1A7FB71237DC021B
:1005460008A190637DE0B4320CD2247E1A7FC412D7
:1005560037DC0208A190637DE0B4330CC2247E1A16
:100566007FD21237DC0208A190637DE0B4340CD24E
:10057600257E1A7FE11237DC0208A190637DE0B484
:10058600350CC2257E1A7FEE1237DC0208A1906375
:100596007DE0FF12001E0208A1906104E0701320A6
:1005A60023077E1A7FFC1237DC9063757421F002F4
:1005B60008A19061047432F0906375E0FFB45104B1
:1005C600C2AF80FEEF645770452023077E1B7F0A6B
:1005D6001237DC90637EE0906331F0E4F52A906395
:1005E60031E0FFE52AC39F40030208A1747F252A54
:1005F600F582E43463F583E0FF90637DE0252A24E9
:10060600ADF582E43461F583EFF0052A80D090637E
:1006160075E0645360030206C22023077E1B7F1524
:100626001237DC90633EE0FF9061B6E06F703C905D
:10063600633FE0FF9061B7E06F7030906340E0FF8A
:100646009061B8E0B50724906341E0FF9061B9E09E
:10065600B50718906342E0FF9061BAE0B5070C90C9
:100666006343E0FF9061BBE06F6016906375742191
:10067600F03023030208A17E1B7F241237DC020818
:10068600A1E4F52AE4F56EAF2AFE74AD252AF582BB
:10069600E43461F583E0FD124898052AE52AC394FF
:1006A600FE40E1C2AFE4907FF0F0A3F0907FFD74CE
:1006B600AAF0A374FFF0A37455F080FE906375E072
:1006C600644F704C90637DE0F528A3E0F529E52999
:1006D6004528700A2023077E1B7F2D1237DC202336
:1006E600077E1B7F341237DCE4F52A747F252AF552
:1006F60082E43463F583E0852982852883F0052921
:10070600E52970020528052AE52AB480DE0208A13B
:10071600906375E0FFB4452190637DE0FDA3E09012
:100726007FF0CDF0A3EDF0C2AF907FFD74AAF0A3E9
:1007360074FFF0A37455F080FEEF64656003020851
:10074600AA90637DE0FFA3E0907FF0CFF0A3EFF0E7
:10075600E4F528F529D3907FF1E09529907FF0E024
:1007660095284020E4F56E2529FFE5283401FE850D
:100776002982852883E0FD1248980529E52970021B
:10078600052880D17E1B7F36124093EF4E602012E3
:100796000003906344EFF0120003906345EFF012FC
:1007A6000003906346EFF0120003906347EFF07E7C
:1007B6001B7F3C124093EF4E602012000390634D66
:1007C600EFF012000390634EEFF012000390634FB8
:1007D600EFF0120003906350EFF07E1B7F42124051
:1007E60093EF4E6020120003906351EFF012000366
:1007F600906352EFF0120003906353EFF012000380
:10080600906354EFF07E1B7F48124093EF4E6020BA
:1008160012000390633AEFF012000390633BEFF08F
:1008260012000390633CEFF012000390633DEFF07B
:100836007E1B7F4E124093EF4E60201200039063A2
:1008460036EFF0120003906337EFF0120003906367
:1008560038EFF0120003906339EFF0E4F52AE4F57F
:100866006EE52A2401FFE433FE7436252AF582E478
:100876003463F583E0FD124898052AE52AC39443BC
:1008860040DCC2AFE4907FF0F0A3F0907FFD74AA45
:10089600F0A374FFF0A37455F080FE7E637F757D30
:0408A60008123F8570
:0108AA00222B
:1047A000AE07EEC39430400BEED394395005EE249F
:1047B000D0FF22EEC39461400BEED394665005EE19
:1047C00024A9FF22EEC39441400BEED3944650053A
:0847D000EE24C9FF22AF06220E
:10493E009062ADE004F070069062ACE004F090621C
:0A494E00ACE0FEA3E0FF12490422D2
:1000030012493E1247A0EFC454F0FEC00612493E07
:080013001247A0D0E02FFF22EC
:10446600E4906A25F012493E906A26EFF0C3943034
:104476004018E0FFD394395011906A25E02405F5E1
:1044860082E43461F583EFF08011906A25E024051B
:10449600F582E43461F583E4F0800C906A25E0044B
:1044A600F0E0D3940840BE752F00753000753100DA
:0C44B600E4F5327B017A617905122BB32A
:0144C20022D7
:044093008E2D8F2EB1
:104097009062ACE4F0A374FFF012493EEF606EF457
:1040A700606B852E82852D83E493B507EC752F0110
:1040B700E52E252FF582E4352DF583E493602590D1
:1040C70062ADE0252FFF9062ACE03400FE12490498
:1040D700E52E252FF582E4352DF583E493B5070406
:1040E700052F80CCE52E252FF582E4352DF583E4C9
:1040F7009370A6E52F24FFFFE434FFFE9062ADE046
:104107002FF09062ACE03EF07E007F0122E4FEFFDC
:014117002285
:103C2F007E1B7F54124093EF4E70037F01227E1B49
:103C3F007F57124093EF4E600C12493EEF24D02471
:103C4F00FF92278002D2277E1B7F5D124093EF4E9B
:103C5F00600C12493EEF24D0906681F08005E4900D
:103C6F006681F07E1B7F63124093EF4E600C12490A
:103C7F003EEF24D090668BF08005E490668BF07E4B
:103C8F001B7F69124093EF4E600C12493EEF24D018
:103C9F0024FF92198002C21990633E63A2019066BD
:103CAF007B63A2017F061228EE30193B7E1B7F6FCC
:103CBF00124093EF4E603012000390667BEFF012CC
:103CCF00000390667CEFF012000390667DEFF01218
:103CDF00000390667EEFF012000390667FEFF01204
:0A3CEF000003906680EFF07F0022D2
:10462300906576E0C3947C40027F0A906576E0FE55
:1046330004F074B42EF582E43462F583EFF0BF0A1C
:1046430027906576E0FF04F074B42FF582E43462BA
:10465300F583E4F0906576E0FF1241189065767477
:0946630008F09062B5E004F022B9
:10451F009080007480F090633663A201F583F5827A
:10452F0063A2017F081228EE90633E63A201908080
:10453F008863A2017F0A1228EE9080927407F0A37D
:10454F0074D0F0A37406F0906348E0FF9080B1F050
:10455F009080E1EFF09080957455F0A3F09080007B
:0A456F007401F090800974F0F0224E
:10439A00908009E04410F09080A0E070609080A1C5
:1043AA007482F09080A874FFF0A3F0A3F0A3F07FCA
:1043BA00039080AEEFF0A374CBF09080007402F00B
:1043CA00906AA512249E00000000906AA5E09080E1
:1043DA0040F0906AA6E0908041F0906AA7E0908051
:1043EA0042F0906AA8E0908043F0A3E4F0A3F0A31F
:0D43FA00F0A3F0908018F0A3F0A3F0A3F062
:014407002292
:1044C300908009E04440F09080D17482F07F0390A3
:1044D30080DEEFF0A374CCF09080027402F0906A57
:1044E300A912249E00000000906AA9E0908058F071
:1044F300906AAAE0908059F0906AABE090805AF0FD
:10450300906AACE090805BF0A3E4F0A3F0A3F0A387
:0B451300F0908030F0A3F0A3F0A3F0C4
:01451E00227A
:10432000908009E04420F09080B8E0706C9080B9F3
:104330007482F07F039080C6EFF07FCDA3EFF07F13
:10434000039080C4EFF0A374CDF09080C074FFF0B0
:10435000A3F0A3F0A3F09080017402F0906AAD1274
:10436000249E00000000906AADE090804CF0906ABE
:10437000AEE090804DF0906AAFE090804EF0906A91
:10438000B0E090804FF0A3E4F0A3F0A3F0A3F0908E
:094390008024F0A3F0A3F0A3F0D7
:014399002201
:10419D008C288D29A907EAFDE975F018A424ACFF38
:1041AD00E5F034808F82F583EDF0EBFDE975F018C5
:1041BD00A4FFAEF024ACFBEE34808B82F583A3ED2F
:1041CD00F08529828C83E0FDEF24A8FFEE3480FE7C
:1041DD008F82F583EDF08529828C83A3E08F828E0B
:1041ED0083A3F0852982852883A3A3E0FDE975F0DB
:1041FD0018A424A8FFE5F03480FE8F82F583A3A3D5
:10420D00EDF08529828C83A3A3A3E08F828E83A3F7
:04421D00A3A3F02245
:063F85008D2DAB07AA061A
:103F8B00908000E030E5079065787401F022906A2C
:103F9B00A5E0FCA3E0FDA3E0FEA3E0F5318E308DA0
:103FAB002F8C2EAE02AF038E838F8263A201E5307E
:103FBB00540744C0F58385318263A201AF2D1229CA
:103FCB0060E4FCFDFEE531252DF531EE3530F530A5
:103FDB00ED352FF52FEC352EF52E908040E52EF09C
:103FEB00A3E52FF0A3E530F0A3E531F0908000744A
:103FFB0020F0AF31AE30AD2FAC2E906AA5122492CB
:01400B002292
:06400C008D28AB07AA0697
:10401200908002E030E5079065787403F022906AA0
:10402200A9E0FCA3E0FDA3E0FEA3E0F52C8E2B8D1E
:104032002A8C29AE02AF038E838F8263A201E52B05
:10404200540744D0F583852C8263A201AF2812293C
:1040520060E4FCFDFEE52C2528F52CEE352BF52B36
:10406200ED352AF52AEC3529F529908058E529F015
:10407200A3E52AF0A3E52BF0A3E52CF090800274CF
:1040820020F0AF2CAE2BAD2AAC29906AA912249253
:01409200220B
:023DB9008F2851
:103DBB00908001E030E5099065787402F07F002275
:103DCB00906AADE0FCA3E0FDA3E0FEA3E0F52C8E32
:103DDB002B8D2A8C2990667B63A201E52B5407441B
:103DEB00C8F583852C8263A2017F06122976E52C08
:103DFB002406F52CE4352BF52BE4352AF52AE4358E
:103E0B0029F52990657963A201E52B540744C8F580
:103E1B0083852C8263A201AF28122976E4FCFDFE78
:103E2B00E52C2528F52CEE352BF52BED352AF52A2F
:103E3B00EC3529F52990804CE529F0A3E52AF0A370
:103E4B00E52BF0A3E52CF09080017420F0AF2CAEA5
:0D3E5B002BAD2AAC29906AAD122492AF283D
:013E68002237
:1036D8009081E0E0F5280528052805280528052813
:1036E80005280528052805280528908010E0F52BD1
:1036F800A3E0F52CA3E0F52DA3E0F52E9081E1E001
:10370800F528052805280528052805280528052859
:10371800052805280528908014E0F52FA3E0F5304A
:10372800A3E0F531A3E0F532E531B52D08E532B572
:103738002E037F0022E4F528E531540744E0F583A1
:1037480085328263A20190637563A2017F08122902
:10375800A690637763A2019062AE63A2017F06120E
:1037680028EE906375E0F529A3E0F52AE4F52890A2
:103778006375E0702AA3E024F8F528E5315407447E
:10378800E0F58385328274082582F582E43583F575
:103798008363A20190637563A201AF281229A6AEC4
:1037A80029E4FCFDE532252AF532E5313EF531ED17
:1037B8003530F530EC352FF52F908014E52FF0A338
:1037C800E530F0A3E531F0A3E532F09080007440D5
:0337D800F0AF2827
:0137DB0022CB
:102D57009081E6E0F5280528052805280528052897
:102D670005280528052805280528908028E0F52B43
:102D7700A3E0F52CA3E0F52DA3E0F52E9081E7E085
:102D8700F5280528052805280528052805280528E4
:102D970005280528052890802CE0F52FA3E0F530BD
:102DA700A3E0F531A3E0F532E4F528E531B52D0AC6
:102DB700E532B52E05C220022EC3E531540744F093
:102DC700F58385328263A20190637563A2017F0850
:102DD7001229A6906375E0F529A3E0F52AE52A45AF
:102DE7002970099080027410F07F0022906682E0BB
:102DF700FFF46030906377E06F6003022E8A90667D
:102E070083E0FF906378E06F7079906684E0FF90CD
:102E17006379E06F706D906685E0FF90637AE06F8D
:102E27006031805F906377E0906682F0906378E02E
:102E3700906683F0906379E0906684F090637AE01F
:102E4700906685F090637BE0FFA3E0906349CFF045
:102E5700A3EFF0906375E0702AA3E024F8F528E566
:102E670031540744F0F58385328274082582F58250
:102E7700E43583F58363A20190637563A201AF28EC
:102E87001229A6AE29E4FCFDE532252AF532E53103
:102E97003EF531ED3530F530EC352FF52FAF2EAE51
:102EA7002DAD2CAC2BAB32AA31A930A82FD31224CD
:102EB7008140099080027410F07F002290802CE5F9
:102EC7002FF0A3E530F0A3E531F0A3E532F09080D1
:062ED700027440F0AF2878
:012EDD0022D2
:1031E1009081E3E0F528052805280528052805280C
:1031F1000528052805280528052890801CE0F52BC1
:10320100A3E0F52CA3E0F52DA3E0F52E9081E4E0F9
:10321100F528052805280528052805280528052855
:10322100052805280528908020E0F52FA3E0F5303A
:10323100A3E0F531A3E0F532E4F528E531B52D0A37
:10324100E532B52E05C221023337E531540744E892
:10325100F58385328263A20190600463A2017F0E2F
:103261001229BC906004E0F529A3E0F52A90600CD6
:10327100E0FFF4604A90667BE0FEEF6E7079A3E0B8
:10328100FF90600DE06F706F90667DE0FF90600EC3
:10329100E06F706390667EE0FF90600FE06F7057A3
:1032A10090667FE0FF906010E06F704B906680E069
:1032B100FF906011E06F703FE4906013F080089020
:1032C100601374FFF0D2D9906004E0702AA3E02467
:1032D100F2F528E531540744E8F583853282740E0E
:1032E1002582F582E43583F58363A201906004634E
:1032F100A201AF281229BCAE29E4FCFDE532252A42
:10330100F532E5313EF531ED3530F530EC352FF55F
:103311002FAF2EAE2DAD2CAC2BAB32AA31A930A8DC
:103321002FD31224815006E52A4529700990800186
:103331007410F07F0022908020E52FF0A3E530F09B
:10334100A3E531F0A3E532F09080017440F0AF289D
:013351002259
:0437DC008E2D8F2E71
:1037E000908000E030E5079065787401F022906ADF
:1037F000A5E0FCA3E0FDA3E0FEA3E0F5348E338D4D
:10380000328C31E534FFE5335407FEE42FF530EE1A
:1038100034C0F52F853082F5837423F00530E53010
:103820007002052F532FC7F582852F83740AF00588
:1038300030E5307002052F532FC790633E63A2011D
:10384000852F8385308263A2017F0612296074066A
:103850002530F530E4352FF52F852D83852E8263B5
:10386000A201852F8385308263A201122944E4FCE2
:10387000FDFE906AA5E0F8A3E0F9A3E0FAA3E02F2B
:10388000FFEE3AFEED39FDEC38FCEF2408FFE43E94
:10389000FEE43DFDE43CFC906AA5122492906AA5EA
:1038A000E0908040F0906AA6E0908041F0906AA796
:1038B000E0908042F0906AA8E0908043F090800011
:0338C0007420F081
:0138C30022E2
:0A35D1008E308F318C328D338B3435
:1035DB00908000E030E5079065787401F022906AE6
:1035EB00A5E0FCA3E0FDA3E0FEA3E0F53A8E398D48
:1035FB00388C37E53AFFE5395407FEE42FF536EE04
:10360B0034C0F535853682F5837423F00536E536FF
:10361B00700205355335C7F582853583740AF0057D
:10362B0036E536700205355335C790633E63A2010C
:10363B0085358385368263A2017F06122960740665
:10364B002536F536E43535F535853083853182639E
:10365B00A20185358385368263A2011229448F3BF3
:10366B00EF2536F536E43535F535E534601785321B
:10367B008385338263A20185358385368263A201FC
:10368B00AF34122960E53B24082534F534FFE4FC04
:10369B00FDFEE53A2FF53AEE3539F539ED3538F5CE
:1036AB0038EC3537F537908040E537F0A3E538F047
:1036BB00A3E539F0A3E53AF09080007420F0AF3A1F
:0C36CB00AE39AD38AC37906AA5122492DD
:0136D70022D0
:0639A5008E298F2A8D2BF4
:1039AB00908000E030E5079065787401F022906A12
:1039BB00A5E0FCA3E0FDA3E0FEA3E0F5318E308D86
:1039CB002F8C2EE531FFE5305407FEE42FF52DEE5D
:1039DB0034C0F52C852D82F5837423F0052DE52D50
:1039EB007002052C532CC7F582852C83EBF0052D2B
:1039FB00E52D7002052C532CC790633E63A2018505
:103A0B002C83852D8263A2017F0612296074062503
:103A1B002DF52DE4352CF52C852983852A8263A27F
:103A2B0001852C83852D8263A201AF2B1229607433
:103A3B0008252BF52BFFE4FCFDFEE5312FF531EED0
:103A4B003530F530ED352FF52FEC352EF52E9080EA
:103A5B0040E52EF0A3E52FF0A3E530F0A3E531F020
:103A6B009080007420F0AF31AE30AD2FAC2E906A49
:043A7B00A5122492DA
:013A7F002224
:024118008F45D1
:10411A00908000E030E5079065787401F022906A9B
:10412A00A5E0FCA3E0FDA3E0FEA3E0F5498E488DDF
:10413A00478C46E549FFE5485407FEE42FFFEE3475
:10414A00C09062B463A201F5838F8263A201AF4576
:10415A00122960E4FCFDFEE5492545F549EE35489E
:10416A00F548ED3547F547EC3546F546908040E58C
:10417A0046F0A3E547F0A3E548F0A3E549F09080AF
:10418A00007420F0AF49AE48AD47AC46906AA5121C
:02419A0024926D
:01419C002200
:0638C4008E288F29AB05E0
:1038CA00908000E030E5079065787401F022906AF4
:1038DA00A5E0FCA3E0FDA3E0FEA3E0F52F8E2E8D6C
:1038EA002D8C2CE52FFFE52E5407FEE42FF52BEE49
:1038FA0034C0F52A852B82F5837423F0052BE52B3A
:10390A007002052A532AC7F582852A83EBF0052B14
:10391A00E52B7002052A90633E63A201852A8385FE
:10392A002B8263A2017F061229607406252BF52BD0
:10393A00E4352AF52A532AC7E528852B82852A8366
:10394A00F0052BE52B7002052A532AC7F582852A32
:10395A0083E529F0052BE52B7002052A532AC7E5D2
:10396A002F240AF52FE4352EF52EE4352DF52DE416
:10397A00352CF52C908040E52CF0A3E52DF0A3E53D
:10398A002EF0A3E52FF09080007420F0AF2FAE2E1A
:0A399A00AD2DAC2C906AA51224920A
:0139A4002200
:0A497700E4FEEEC39F50030E80F82B
:014981002213
:10490400A2AF9228C2AF438E2075D2028F828E83CB
:0C491400E0FFE4F5D2538EDFA22892AF42
:014920002274
:10489800E5D220E0FBA2AF9228C2AF43D2028F82BA
:1048A8008E83EDF075D25063D250A22892AFE5D234
:0348B80020E0FB02
:0148BB0022DA
:1042A200E4FDED2401FFE433FE12490474362DF5DA
:1042B20082E43463F583EFF00DBD3FE6E4FDED24C7
:1042C2007FFFE433FE124904742D2DF582E434613C
:1042D200F583EFF0742D2DF582E43461F583E070FF
:1042E2001B742D2DF582E43461F5837420F0742E55
:1042F2002DF582E43461F583E4F080040DBD80BEC7
:10430200E49061ACF0FDEDFF7E0012490474AD2D26
:0D431200F582E43461F583EFF00DBDFEE9A6
:01431F00227B
:02480D008B2DF1
:10480F00A2AF9228C2AF85A22E53A2FE8E838F82B3
:10481F0005A28C838D8274091229EAE52D53A2FE1D
:10482F0043A2201229EC53A2DF852EA2A22892AF19
:01483F00FF79
:014840002255
:10492100A2AF9228C2AF8C838D82EF1229EA43A2F3
:0C493100201229EC53A2DFA22892AFFF55
:01493D002257
:0248BC008F2843
:1048BE00A2AF9228C2AFE4F5838D8274061229EA64
:1048CE00E52843A2201229EC53A2DFA22892AF7F43
:0148DE0001D8
:0148DF0022B6
:0248E0008F281F
:1048E200A2AF9228C2AFE4F5838D82740A1229EA3C
:1048F200E52843A2201229EC53A2DFA22892AF7F1F
:0149020001B3
:014903002291
:10281300A907E7FFA805EF93C3966008403B74FC44
:102823002FFF80F00F08EF93C3966008402B74FBD3
:102833002FFF80E00F08EF93C3966008401B74FAE4
:102843002FFF80D00F08EF93D3966008400B74F9E5
:102853002FFF80C01F1F1F1F1FEF54FEF80303F736
:10286300E893FC08E893FD08E893FE08E893FF2249
:1028730009E993C39D6008402974FB29F980F10994
:10288300E993C39E6008401A74FA29F980E209E9C2
:1028930093D39F6008400B74F929F980D319191950
:1028A3001919E9C313C313FF22740093F8ECC398F7
:1028B3004024701F740193F8EDC398401970147489
:0E28C3000293F8EEC398400E7009740393F868
:1028D100EFC39840037F00227F0122EDF8E6F00864
:1028E100A3DFFA22EDF8E0F608A3DFFA22E0A36302
:1028F100A201F0A363A201DFF475A2002263A20189
:10290100F0A363A20122E0A363A201F0A363A201E9
:10291100E0A363A201F0A363A201E463A201F0A317
:1029210063A201DFE175A20022E0A363A2016DFEB3
:10293100936CFDEE058393FC158363A201DFEA75B9
:10294100A200227F00E493A363A201F00F600CA315
:10295100E583C2E3F58363A20180EA75A20022E068
:10296100A363A201F0A3E583C2E3F58363A201DFC0
:10297100EE75A20022E0A363A201F0A3E583C2E405
:10298100D2E3F58363A201DFEC75A20022E0A36329
:10299100A201F0A3E58344F8C2E5F58363A201DF58
:1029A100EC75A20022E583C2E3F583E0A363A201F3
:1029B100F0A363A201DFEE75A20022E583C2E4D297
:0A29C100E3F583E0A363A201F0A395
:1029CB0063A201DFEC75A20022E58344F8F583E0F6
:1029DB00A363A201F0A363A201DFEE75A20022F9AB
:1029EB0022C002C004C00612FFF0D006D004D002F1
:0129FB0022B9
:10001E00BF360BD20BE4F54AF54BF566F567BF37E5
:04002E0002C20B22DD
:10440800C2A9438902906A20E0FFF58C8F8A75D98A
:104418000475DA4875DB3175DC4975DD4975DE31BF
:10442800E4F5E9F5F9F5EBF5FB906A1EE060167521
:10443800EC1075ED10E4F5FCF5FD7562087560107B
:10444800756101801375EC8075ED80E4F5FCF5FD70
:0E445800756280F560756110E4F5EEF5FE22E8
:10476700E4FEAF8CEFFD906A1FE07003A3E06D607D
:10477700051244087E01E5D920E2057E02124408AD
:10478700E58920E1051244087E03D28C75D840756F
:08479700B740D2AED2AFAF066D
:01479F0022F7
:0300330002306434
:0B306400C0E0C083C082C0D075D0085F
:10306F00C2AF30DC56C3E5EC95EEC395625012E566
:10307F006125ECF5EC30D70405FC801685FCFC804F
:10308F0011C3E5EC9561F5EC30D70415FC80038591
:10309F00FCFC300B24854B82854A83E590F0054B71
:1030AF00E54B7002054AF582854A83E5EEF0054B44
:1030BF00E54B7002054A534A0FC2DC30D929300B59
:1030CF0024854B82854A83E590F0054BE54B7002D2
:1030DF00054AF582854A83E5EBF0054BE54B700217
:1030EF00054A534A0FC2D930DA69E560700405FC0E
:1030FF008010E56025ECF5EC30D70405FC800385E6
:10310F00FCFC300C4CE54C5480FFE54C25E0F54CB5
:10311F00309702054C200A03634C01303119E54CFE
:10312F0054C06568702BEF7028756308F55E854C89
:10313F004FF54CC231801A0563E563540770125383
:10314F00633FE563131313541F244EF8A64C754CBD
:10315F0000C2DA30DB71E560700405FD8010E560B8
:10316F0025EDF5ED30D70405FD800385FDFDE56404
:10317F00655F6029E55F54077013E55F1313135400
:10318F001F2456F8E6F54D200803634DFFE54D3338
:10319F009296E54D25E0F54D055F535F3FB29230B6
:1031AF000B23854B82854A83E590F0054BE54B70E9
:1031BF0002054AF582854A83E4F0054BE54B700220
:0931CF00054A534A0FC2DBD2AFDE
:0931D800D0D0D082D083D0E032C7
:101B75000ACFEEEFFBF2EAE020EEF2EFF0E0E2EA68
:101B8500E820F1EBE8F8EAEEEC20E4EBE8EDEDEE29
:101B9500E3EE20EFE0EAE5F2E021000A536F6D6520
:101BA50020646174612066726F6D20686F737400C4
:101BB5000ACEF2EFF0E0E2EAE020D2D30A000ACE44
:101BC500F2EFF0E0E2EAE0204F5420EEF220F1E5FA
:101BD500F0E2E5F0E00A000ACEF2EFF0E0E2EAE03A
:101BE50020E7E0EFF0EEF1E020EEF220F1E5F0E2A3
:101BF500E5F0E00A000A536F6D65206461746120A9
:101C050066726F6D206368616E6E656C000A435283
:101C150043206572726F7221000ACFF0E8B8EC209C
:101C2500E8EDF4EEF0ECE0F6E8E8000AD7F3E6EECE
:101C3500E920CACF21000AC6E4E0EB20E8EDF4F381
:101C450020E020F2F3F220F7F2EE2DF2EE20EDE5A2
:101C550020F2EE2E2E2E000ACAE2E8F2E0EDF6E8BA
:101C6500FF20D2D321000ACDE5F220E8EDF4EEF015
:101C7500ECE0F6E8E821000ACFF0E8B8EC20E7E070
:101C8500EFF0EEF1E0000ACDE0F7E0EBEE20EFF04B
:101C9500E8B8ECE0000AC8F1F2E5EAEBEE20E2F084
:101CA500E5ECFF20EEE6E8E4E0EDE8FF20EEF2E209
:101CB500E5F2E0000AC7E0EFF0EEF120E3F0F3EF24
:101CC500EFFB20D2C8D2200020EEF220CACF2000A0
:101CD5000A000ACEF2EFF0E0E2EAE020CED220EDF3
:101CE500E020CACF2000202020CFEEE2F2EEF02047
:101CF500EAEEECE0EDE4FB0A000D0AC8F1F2E5EAD4
:101D0500EBEE20E2F0E5ECFF20EEE6E8E4E0EDE8BE
:101D1500FF20E4EEF1F2E0E2EAE820EFE0EAE5F2A6
:101D2500E0003E2A2C312CCFE0F0E0ECE5F2F0FBB0
:101D350020F1E8EDF5F0EEEDEDEEE3EE20EFEEF05F
:101D4500F2E00A003E4C2C4230312C256C752CD12A
:101D5500EAEEF0EEF1F2FC20EEE1ECE5EDE02C35FB
:101D6500302C3130302C3230302C3330302C363072
:101D7500302C313230302C323430302C3438303055
:101D85000A003E422C4731302C2562752CC8EDE205
:101D9500E5F0F1E8FF20EDE020EFF0E8B8ECE50A2A
:101DA500003E422C4731312C2562752CC8EDE2E509
:101DB500F0F1E8FF20EDE020EFE5F0E5E4E0F7E500
:101DC5000A003E422C4730322C2562752CD3EFF0A9
:101DD500E0E2EBE5EDE8E520EFEEF2EEEAEEEC20F1
:101DE50020285254532D435453290A003E532C475F
:101DF50030332C256C752CC7E0E4E5F0E6EAE020ED
:101E0500F1F2E0F0F2E020EFE5F0E5E4E0F7E828B4
:101E1500ECF1290A003E2A2C312CC0E4E0EFF2E572
:101E2500F020F1E8EDF5F0EEEDEDEEE3EE20EAE081
:101E3500EDE0EBE02E20CFF0EEF2EEEAEEEB200047
:101E4500CAEEECEFE0F120D2CC312E310A00D3C23C
:101E5500D2CA2D3132300A003E422C4B31322C256C
:101E650062752CD3C2D2CA2D3132300A003E422CC3
:101E75004B30342C2562752CD0E5E6E8EC20EFF0EC
:101E8500EEF1EBF3F8EAE820EAE0EDE0EBE020F133
:101E9500E2FFE7E80A003E422C4B31312C25627502
:101EA5002CD0E5E6E8EC20F1E8ECF3EBFFF6E8E80A
:101EB50020CACF0A003E532C4B30312C25732CD130
:101EC500EFE8F1EEEA20CACF0A003E422C4B30384B
:101ED5002C2562752CD3EFF0E0E2EBE5EDE8E5208B
:101EE500D0CA0A003E532C4B30322C25732CCAEE37
:101EF500EB2DE2EE20E3F0F3EFEF20D2C8D20A009B
:101F05003E532C4B30332C25732CCFF0E8EEF0E804
:101F1500F2E5F220CED220EA20C7C3D2C8D20A0009
:101F25003E532C4732302C256C752CC2F0E5ECFF66
:101F350020EEE6E8E4E0EDE8FF20EEF2E2E5F2E08F
:101F450028ECF1290A003C21003C4230313D003C9F
:101F55004731303D003C4731313D003C4730323D53
:101F6500003C4730333D003C4732303D003C4B3070
:101F7500343D003C4B31313D003C4B31323D003C62
:101F85004B30383D003C4B30313D003C4B30323D11
:071F9500003C4B30333D001E
:103CFF0052668D0000000000000000000000000070
:103D0F00000000000060A0697300050002000005BC
:103D1F00000200000500020000050002000005007F
:103D2F00020000050002000005000200000500026D
:103D3F00000005000200000500020000050002005F
:103D4F00000500020000050002000005000200004F
:103D5F00050002000005000200000500020000053A
:103D6F00000200000500020000050002000005002F
:103D7F00020000050002000005000200000500021D
:103D8F00000005000200000500020000050002000F
:103D9F0000050002000005000200000500020000FF
:093DAF00050002000005000200FD
:0100320022AB
:024221008D2CE2
:10422300AA06A907752F018A308931E4F52D1249B1
:104233003E8F2EE52E643C6030E52E642C602AAB65
:104243002FAA30A931E52E12237174012531F531DE
:10425300E43530F530052D12493E8F2EE52E643CB2
:104263006007E52DC3952C40D6E52D7016AB2FAA1C
:1042730030A931742012237174012531F531E435ED
:1042830030F530E52DB52C0C74FF2531F53174FF75
:0E4293003530F530AB2FAA30A931E41223717B
:0142A10022FA
:10472D00301534E4906475F0906971E0FD90647615
:10473D00F090667AE0906477F0A37405F09068705D
:10474D00E0543FF063A20190647963A201AF0512BA
:0A475D0028EEC2157F01227F002222
:1029FC00906A1F74FFF0A374B8F0E4906A1EF09014
:102A0C006A18F0C2131225BEE4F529F528742125A5
:102A1C0028F582E43467F583E0FF6070E529C39400
:102A2C00205069EFB42004052880E2E52975F005F3
:102A3C00A42473F9746935F0FA906A147401F0A344
:102A4C00EAF0A3E9F074212528F9E43467FA7B0154
:102A5C00C0031B8B2F753000753100E4F532D003A9
:102A6C00122BB3906A14E0FBA3E0FAA3E0F9EF1287
:102A7C002371052974212528F582E43467F583E058
:102A8C00FF64206088EF6085052880E8E5297005E3
:102A9C00D213022BAFE4F529F52874C72528F5824B
:102AAC00E43467F583E0FF6073E529C39420506C30
:102ABC00EFB42004052880E2E52975F005A4247301
:102ACC00F9746935F0FA906A147401F0A3EAF0A372
:102ADC00E9F074C72528F9E43467FA7B01C0031BBD
:102AEC008B2F753000753100E4F532D003122BB307
:102AFC00906A14E0FBA3E0FAA3E0F9900003EF1254
:102B0C002383052974C72528F582E43467F583E00F
:102B1C00FF64206085EF6082052880E8E4F529F5E4
:102B2C0028749F2528F582E43466F583E0FF6073F2
:102B3C00E529C39420506CEFB42004052880E2E50D
:102B4C002975F005A42473F9746935F0FA906A14A8
:102B5C007401F0A3EAF0A3E9F0749F2528F9E4349A
:102B6C0066FA7B01C0031B8B2F753000753100E4B6
:102B7C00F532D003122BB3906A14E0FBA3E0FAA356
:102B8C00E0F9900001EF1223830529749F2528F5A5
:102B9C0082E43466F583E0FF64206085EF60820593
:062BAC002880E812440835
:012BB2002200
:1046B0007568C0C20BC207E4F54CC215C212C20233
:1046C000D214F55EF563906A19F09067C4F0906AB1
:1046D0001C7403F030161290671FF0D2319067C53A
:1046E000E09067C4F0D20C8005E490671FF0124799
:0246F00067223F
:1046F200AE07906A13E0FF30E10A6402F0906A1795
:10470200E06429F0906A13E0FF25E0F0906A17E078
:10471200FD30E707906A13E04401F0ED25E0906A6E
:0B47220017F0EE30E704E04401F02245
:023B5900AA07B9
:103B5B00D22CE4FB200105AF021246F29067A1E0E4
:103B6B00FF25E0F0EA30E709E04401F0A22CB39224
:103B7B002C9068F0E004F0E0B4081E9067A1E0859B
:103B8B001682851583F00516E516700205159069EA
:103B9B0072E004F0E49068F0F0EA25E0FA0BBB0861
:103BAB00B3200111A22A302C01B350047F80800274
:103BBB007F001246F29067A1E0FF25E0F0A22BE414
:103BCB0033600F14701B302A189067A1E04401F08A
:103BDB00800FA22A302C01B350079067A1E044015B
:103BEB00F09068F0E004F0200112906A13E0FF30CF
:103BFB00E10A6402F0906A17E06429F09068F0E043
:103C0B00B4081E9067A1E0851682851583F0051612
:103C1B00E51670020515906972E004F0E49068F007
:033C2B00F0C201E3
:013C2E002273
:0234BD00AA075C
:1034BF00E4FB200138906A13E0FF30E10A6402F068
:1034CF00906A17E06429F0906A13E0FF25E0F0900E
:1034DF006A17E0FE30E707906A13E04401F0EE252B
:1034EF00E0906A17F0EA30E704E04401F09068F0EA
:1034FF00E004F0E024F8602914605A8000EA30E715
:10350F000E906A1AE04401F0A205B392058007906D
:10351F006A1AE054FEF0906A1AE0FF25E0F00235D7
:10352F00C1EA30E70E906A1AE04401F0A205B392A7
:10353F00058007906A1AE054FEF0906A1AE085142D
:10354F0082851383F00514E51470020513906971D9
:10355F00E004F0805D300626D21130101E906A1301
:10356F00E0FF30E10A6402F0906A17E06429F090FE
:10357F006A17E0FF906A13E04FFF227F00223005A9
:10358F0015EA20E724D206906A1AE0B42004D2107C
:10359F008017C2108013EA30E70FD206906A1AE044
:1035AF00B42004D2108002C210C201D205E4906888
:1035BF00F0F0EA25E0FA0BEB640860030234C17FF8
:0135CF0000FB
:0135D00022D8
:0245D100A90738
:1045D300E4906972F0752968752A4875156875162F
:1045E300F1852A82852983E044C0F0E49068F0F0E5
:1045F300FCECC399501A852A82852983E0FFC22ADD
:10460300C22B123B59052AE52A700205290C80E1C9
:0F461300D22AC22BE4FF123B597515687516F1B8
:014622002275
:023352008F28C2
:103354003002030234ABD21774FC2528F52813136A
:1033640013541FFF2528FFE433CF2402CF3400FE7B
:10337400C3EF9420EE64809480401130250B7E1BB3
:103384007F75E4FBFDFC1235D1D21422752B018527
:10339400152C85162D906972E0F52EE4F0906A13D1
:1033A400F0906A17F030250D7E1B7FA07C637D7939
:1033B400AB281235D1752963752A7974782528F5D7
:1033C40082E43463F583E0B42003D38001C39229FB
:1033D40015287515677516A3852A82852983E04407
:1033E400C0F09068F0E0F52FE4F0D201FCECC39556
:1033F40028501A852A82852983E0FFC22AC22B120B
:103404003B59052AE52A700205290C80E03029621F
:10341400D22AC22B7F20123B59E4FCE4FF1246F26D
:103424000CBC09F7906A13E0FF30E10A6402F090E3
:103434006A17E06429F0906A17E0FF30E003D38054
:1034440001C39228EFC313906A17F0906A13E03017
:10345400E009906A17E04480F08007906A17E0540E
:103464007FF0D201906A17E0FFA228922AD22B1291
:103474003B59D22AC22BE4FF123B59D20290697203
:10348400E09067C3F0906972E52EF0852C15852DC8
:10349400167517017518677519A39068F0E52FF074
:1034A400906A1C7403F022906A1CE0600214F0908D
:0834B4006A1CE070031246B02F
:0134BC0022ED
:103A8000E4FF0F2405F582E43461F5837405F00F3B
:103A900074052401F582E43461F583E4F0752801AE
:103AA000752966752A92FEAB28E52A152AAA29707F
:103AB000021529F91222F8FDAC070F74052CF582C6
:103AC000E43461F583EDF00EBE04DC752801752940
:103AD00066752A96E4FEAB28E52A152AAA29700203
:103AE0001529F91222F8FDAC070F74052CF582E4B4
:103AF0003461F583EDF00EBE04DC7528017529668E
:103B0000752A9AE4FEAB28E52A152AAA297002151F
:103B100029F91222F8FDAC070F74052CF582E43464
:103B200061F583EDF00EBE04DC752801752966751C
:103B30002A9EE4FEAB28E52A152AAA297002152937
:103B4000F91222F8FDAC070F74052CF582E43461FC
:083B5000F583EDF00EBE04DC6C
:013B5800224A
:0F496800C211C207C206200003C20C22D20C22C9
:0247D8008F2927
:1047DA00E4F52AE52A75F005A42473F9746935F01D
:1047EA00FA7B01906A14EBF0A3EAF0A3E9F0122233
:1047FA00F8B52905E52A04FF22052AE52AB420D3BB
:02480A007F002D
:01480C002289
:05498D001FEF70FC2289
:10487000AE07EDD39400401FEE30E703D38001C3B1
:104880009291D2907F0A12498DC2907F0A12498D6F
:07489000EE25E0FE1D80DBB8
:0148970022FE
:02484100AC07C2
:10484300AB04EB33333354F8FB5303C04303156317
:1048530003FFAF037D08124870AB04EBC454F0FBB5
:0C486300530370AF037D04124870D29024
:01486F002226
:1008AB00300B2DC3E54B9567FFE54A9566FED3EFFD
:1008BB009440EE940040197B087D40AF67AE661202
:1008CB0039A5E5672440FFE43566540FF5668F675D
:1008DB00201B0302104E301A0AC21A9067C4E06044
:1008EB000214F090671FE0B4090050229008FEF844
:1008FB0028287302091F020A25020A25020B2F0260
:10090B000E4B020B2F020FE002100C02102FE49083
:10091B00671FF02230161390671F7403F0D23190CB
:10092B0067C5E09067C4F0D20C22200203020A08CC
:10093B009067C3E0906972F0C202E4F52890697287
:10094B00E0FFE528C39F5026AB17AA18A91912225E
:10095B00F8FE74482528F582E43468F583EEF074CC
:10096B00012519F519E43518F518052880CF7515EB
:10097B00687516488515118516128F103009047F7E
:10098B000880027F0190671FEFF085168285158323
:10099B00A3E0547FFF64706003BF381F9067A2749D
:1009AB0006F0D20420250302104E7E1B7FB5906902
:1009BB0072E0FBAD16AC151235D12285168285156A
:1009CB0083A3E0547FFFBF281A3025107E1B7FC303
:1009DB00906972E0FBAD16AC151235D19067A2741D
:1009EB0005F0223025107E1B7FDC906972E0FBAD99
:1009FB0016AC151235D19067A27403F02230001398
:100A0B0090671F7405F0D2319067C5E09067C4F012
:100A1B00D20C2290671F7404F022201203020ADB0F
:100A2B00E564655F604DE56424085438FFE55F5469
:100A3B00386F60047E0180027E00906972E0600472
:100A4B007D0180027D00EE5D700302104E851682E3
:100A5B00851583E0FEE564131313541F2456F8A683
:100A6B00068F640516E51670020515906972E01481
:100A7B00F080B39067A2E064066038906693E0FC68
:100A8B00A3E0FDA3E0FEA3E0FFE4FAF9F8EF2401F5
:100A9B00FFEA3EFEE93DFDE83CFC90669312249292
:100AAB00D20CE4F54CD231D2B19067C5E09067C45B
:100ABB00F080069067C47441F0301704D214C2174B
:100ACB00C212200902C2909067A2E090671FF02229
:100ADB0030B10B300F08906720E09067C4F0C2B1C3
:100AEB00300F0C30B0099067C4E0600302104E85E4
:100AFB001682851583E0FFE564131313541F2456E8
:100B0B00F8A607E56424085438F5640516E5167055
:100B1B00020515906972E014F0D21230090302102D
:100B2B004ED29022200703020DB8E5635438655E60
:100B3B00700302104EE55E24085438F55E13131350
:100B4B00541F244EF8E6906847F0200623E0FF126E
:100B5B0034BD8F28906971E0D39480500302104EFE
:100B6B0090671F7407F09067C47432F012496822C3
:100B7B00200902C29130002E906971E014F0D21559
:100B8B0090671F7407F09067C47432F012496820A5
:100B9B00250302104E7E1B7FFA7C687D7090697175
:100BAB00E0FB1235D122201003020C9A90671FE054
:100BBB0064036003020C9A906847E0FF1234BD8F08
:100BCB0028201103020B35E528603CC21530251097
:100BDB007E1C7F127C687D70906971E0FB1235D1B1
:100BEB00906697E0FCA3E0FDA3E0FEA3E0FFE4FA30
:100BFB00F9F8EF2401FFEA3EFEE93DFDE83CFC90ED
:100C0B006697122492807820160C906848E0FF902B
:100C1B006870E06F7056906971E024FEF0D2153069
:100C2B00250F7E1C7F1E7C687D70E02402FB123535
:100C3B00D1300E11906871E0B4F00A906971E02424
:100C4B00FD906872F090668FE0FCA3E0FDA3E0FEE0
:100C5B00A3E0FFE4FAF9F8EF2401FFEA3EFEE93DD9
:100C6B00FDE83CFC90668F12249280133025107E99
:100C7B001C7F307C687D70906971E0FB1235D190E0
:100C8B00671F7407F09067C47432F01249682290A2
:100C9B00671FE0640370233025107E1C7F3B7C684C
:100CAB007D70906971E0FB1235D190671F7407F06E
:100CBB009067C47432F01249682230042AC204D2FD
:100CCB0015906971E014F030250D7E1C7F5C7C68FB
:100CDB007D70E0FB1235D190671F7407F09067C4ED
:100CEB007432F012496822906848E0FF906870E017
:100CFB006F60233025107E1C7F307C687D7090697F
:100D0B0071E0FB1235D190671F7407F09067C474C4
:100D1B0032F012496822906849E0FF906871E06FE9
:100D2B00702E3025107E1C7F6B7C687D70906971F6
:100D3B00E0FB1235D1301308D215906971E014F035
:100D4B0090671F7407F09067C47432F012496822E1
:100D5B003025117E1C7F7C7C687D70906971E0145E
:100D6B00FB1235D120160330131690671F7407F052
:100D7B009067C47432F0D215906971E014F0802939
:100D8B00906870E0906848F0906871E0906849F066
:100D9B00906872E090684AF07F031245D190671F0C
:100DAB007401F09067A27403F01249682220313667
:100DBB0030250B7E1C7F8BE4FBFDFC1235D1E490C0
:100DCB0067C4F0D207200902D291E4906971F090C8
:100DDB006A17F0906A13F0D2059068F0F0D20175A3
:100DEB00136875147022300009300206E490671FF7
:100DFB00F02230160302104E9067C4E0600302101D
:100E0B004E30250A7E1C7F9AFBFDFC1235D1906675
:100E1B009BE0FCA3E0FDA3E0FEA3E0FFE4FAF9F8FE
:100E2B00EF2401FFEA3EFEE93DFDE83CFC90669BAA
:100E3B0012249290671F7407F09067C47432F022EB
:100E4B0030130D90671F7407F09067C47432F02253
:100E5B00906A19E004F0E0C394204002E4F0906A39
:100E6B0019E075F005A42473F9746935F0FA7B0168
:100E7B00906A14EBF0A3EAF0A3E9F01222F8FF70EA
:100E8B0003020FCD906A14E0FBA3E0FAA3E0F99004
:100E9B000002740112233E900001122311FE9000F8
:100EAB0002122311C39E5003020F6D906A14E0FBD4
:100EBB00A3E0FAA3E0F9900002E41223839000046C
:100ECB00740112233E900003122311FE90000412B2
:100EDB002311D39E4013906A14E0FBA3E0FAA3E026
:100EEB00F99000047401122383906A14E0FBA3E0D1
:100EFB00FAA3E0F9906848EFF0A37410F0900004A7
:100F0B0012231190684AF09067A27403F0FF124508
:100F1B00D1202503020FBE7E1C7FB9906A14E0A37B
:100F2B00E0FAA3E02404F9E43AFCAD017B011235AD
:100F3B00D17F1E1249777E1C7FCD906A14E0A3E00F
:100F4B00FAA3E0AC02FD7B011235D17F1E1249776B
:100F5B007E1C7FD57C687DF1906972E0FB1235D1E8
:100F6B008051906A14E0FBA3E0FAA3E0F91222F897
:100F7B00906848F0A37450F0E4A3F09067A2740556
:100F8B00F07F031245D130252A7E1C7FD7906A143F
:100F9B00E0A3E0FAA3E0AC02FD7B011235D17F1E8A
:100FAB001249777E1C7FD57C687DF1906972E0FBDE
:100FBB001235D13009047F0880027F0190671FEF43
:100FCB00F022906A1974FFF090671F7407F0906716
:100FDB00C47432F0229067C4E0706830250A7E1C1E
:100FEB007FEBFBFDFC1235D190671F7401F090670E
:100FFB00A27405F0851115851216906972E510F033
:10100B00223015169067C4E070397E1C7FFEFBFD05
:10101B00FC1235D1E490671FF022E49067C4F09086
:10102B00671FF022851682851583E0543FFF124718
:10103B00D88F28E528D39400400312484190671FAE
:03104B007401F03D
:01104E00227F
:0B498200301405C2147F01227F0022C8
:03499200C2AE2290
:102EDE00906A1EE0601EA3E0FEA3E0FFC3E49FFF26
:102EEE00E49EFEAB07FAE4F9F8FF7EC27D01FC1208
:102EFE00466C801E906A1FE0FEA3E0FFC3E49FFFB6
:102F0E00E49EFEAB07FAE4F9F87F207E1CFDFC126E
:102F1E00466C8F308E2F8D2E8C2D7BFF7A1D792750
:102F2E00121FFE7BFF7A1D7949853037852F368536
:102F3E002E35852D34121FFE7BFF7A1D7987A20A4E
:102F4E00E433F534121FFE7BFF7A1D79A6A208E446
:102F5E0033F534121FFE7BFF7A1D79C7A20FE433BF
:102F6E00F534121FFE7BFF7A1D79F1906720E07514
:102F7E00F00AA4FFAEF0E48F378E36F535F5341235
:102F8E001FFE7534FF75351E75361A7B017A6A7908
:102F9E0021121FF8200E147534FF75351E75364537
:102FAE007B017A6A792112457980127534FF753565
:102FBE001E7536537B017A6A79211245797B017A27
:102FCE006A7921121FFE7BFF7A1E795DA20EE43311
:102FDE00F534121FFE7BFF7A1E7972A216E433F5CA
:102FEE0034121FFE7BFF7A1E799BA200E433F53468
:102FFE00121FFE7534017535677536217BFF7A1EFB
:10300E0079BA121FFE7BFF7A1E79CFA209E433F53F
:10301E0034121FFE7534017535677536C77BFF7A1E
:10302E001E79E9121FFE75340175356675369F7B64
:10303E00FF7A1F7905121FFE7BFF7A1F7925906795
:10304E00C5E075F00AA4FFAEF0E48F378E36F53585
:05305E00F534121FFE15
:01306300224A
:1025BE007E1F7F4B124093EF4E70037F01227E1FD2
:1025CE007F4E124093EF4E700302266512446690C2
:1025DE006A21122492E4FFFEFDFC906A21E0F8A32A
:1025EE00E0F9A3E0FAA3E0FBC31224816025906A10
:1025FE0021E0F8A3E0A3E0A3E0E47F207E1CFDFC35
:10260E001223E1122473906A1FEEF0A3EFF0E49010
:10261E006A1EF0E47FB07E04FDFC906A21E0F8A310
:10262E00E0F9A3E0FAA3E0FBD31224814038906ACC
:10263E001E7401F0906A21E0F8A3E0A3E0A3E07F0E
:10264E00007EC27D017C001223E1122473906A1F6A
:10265E00EEF0A3EFF0800F906A1F74FFF0A374B832
:10266E00F0E4906A1EF07E1F7F54124093EF4E608E
:10267E000C12493EEF24D024FF920A8002C20A7E39
:10268E001F7F5A124093EF4E600C12493EEF24D03A
:10269E0024FF92088002C2087E1F7F60124093EFD3
:1026AE004E600C12493EEF24D024FF920F8002C2DE
:1026BE000F7E1F7F66124093EF4E6013124466E446
:1026CE007B0AFAF9F81223E1906720EFF08005E417
:1026DE00906720F07E1F7F6C124093EF4E601112B8
:1026EE004466E47B0AFAF9F81223E19067C5EFF02D
:1026FE009067C5E07003740AF07E1F7F72124093DC
:10270E00EF4E600C12493EEF24D024FF9216800249
:10271E00C2167E1F7F78124093EF4E600C12493E18
:10272E00EF24D024FF92008002C2007E1F7F7E1213
:10273E004093EF4E600C12493EEF24D024FF920ED0
:10274E008002C20E7E1F7F84124093EF4E600C12E9
:10275E00493EEF24D024FF92098002C209E4F52AF3
:10276E007E1F7F8A124093EF4E600B7E677F217D26
:10277E0080124221801EAF2A052A74212FF582E491
:10278E003467F5837420F07421252AF582E43467CA
:10279E00F583E4F0E4F52A7E1F7F90124093EF4E0E
:1027AE00600B7E677FC77D80124221801EAF2A0597
:1027BE002A74C72FF582E43467F5837420F074C74A
:1027CE00252AF582E43467F583E4F0E4F52A7E1FCA
:1027DE007F96124093EF4E600B7E667F9F7D801238
:1027EE004221801EAF2A052A749F2FF582E434669B
:1027FE00F5837420F0749F252AF582E43466F58300
:04280E00E4F07F0073
:0128120022A3
:103F050002104FE493A3F8E493A34003F68001F273
:103F150008DFF48029E493A3F85407240CC8C333BD
:103F2500C4540F4420C8834004F456800146F6DF8C
:103F3500E4800B0102040810204080903CF9E47EE7
:103F4500019360BCA3FF543F30E509541FFEE49381
:103F5500A360010ECF54C025E060A840B8E493A348
:103F6500FAE493A3F8E493A3C8C582C8CAC583CA73
:103F7500F0A3C8C582C8CAC583CADFE9DEE780BE2B
:013DB800000A
:1022F800BB010689828A83E0225002E722BBFE02E4
:09230800E32289828A83E4932216
:10231100BB010CE58229F582E5833AF583E0225081
:1023210006E92582F8E622BBFE06E92582F8E222CB
:0D233100E58229F582E5833AF583E49322E5
:10233E00BB010FF8E58229F582E5833AF583E028A3
:10234E00F0225009C58229F8E58226F622BBFE0945
:10235E00C58229F8E22582F222F8EA2583F583E97F
:03236E009328228F
:10237100BB010689828A83F0225002F722BBFE014B
:02238100F32245
:10238300F8BB010DE58229F582E5833AF583E8F090
:10239300225006E92582C8F622BBFE05E92582C83C
:0223A300F22224
:1023A50075F008758200EF2FFFEE33FECD33CDCCEF
:1023B50033CCC58233C5829BED9AEC99E582984072
:1023C5000CF582EE9BFEED9AFDEC99FC0FD5F0D64F
:1023D500E4CEFBE4CDFAE4CCF9A88222B800C1B979
:1023E5000059BA002DEC8BF084CFCECDFCE5F0CBB7
:1023F500F97818EF2FFFEE33FEED33FDEC33FCEBF0
:1024050033FB10D703994004EB99FB0FD8E5E4F9AA
:10241500FA227818EF2FFFEE33FEED33FDEC33FC97
:10242500C933C910D7059BE99A4007EC9BFCE99A8B
:10243500F90FD8E0E4C9FAE4CCFB2275F010EF2FD0
:10244500FFEE33FEED33FDCC33CCC833C810D707D0
:102455009BEC9AE899400AED9BFDEC9AFCE899F80B
:0E2465000FD5F0DAE4CDFBE4CCFAE4C8F9229E
:10466C00C2D5E830E70FB2D5E4C39BFBE49AFAE479
:10467C0099F9E498F8EC30E717B2D51246A2122358
:10468C00E1E4C39BFBE49AFAE499F9E498F880031B
:10469C001223E130D50DE4C39FFFE49EFEE49DFDA3
:0446AC00E49CFC226C
:0E247300C3E49FFFE49EFEE49DFDE49CFC227A
:10248100EB9FF5F0EA9E42F0E99D42F0E89C45F0B1
:012491002228
:0C249200ECF0A3EDF0A3EEF0A3EFF022BD
:10249E00A8828583F0D083D0821224B51224B5127F
:1024AE0024B51224B5E473E493A3C583C5F0C583A4
:1024BE00C8C582C8F0A3C583C5F0C583C8C582C888
:0124CE0022EB
:101F9C00E5402434F8E60540227831302F027834BD
:101FAC00E475F00112251E0222F82028EB7F2ED2B8
:101FBC00288018EF540F2490D43440D4FF302C0BCD
:101FCC00EF24BFB41A0050032461FFE541600215F1
:101FDC00410544E54470020543302F0D7831E4751A
:101FEC00F00112251EEF0223710246237403D22F37
:101FFC008003E4C22FF5408B318A328933E4F541FA
:10200C00F543F544E54160077F20121FD780F57535
:10201C0042FFC229C228C22AC22BC22DC22EC230F4
:10202C00121FA5FF700D302F057F00121FE8AF4463
:10203C00AE4322B4255FC2D5C22C121FA5FF24D0FB
:10204C00B40A00501A75F00A784130D50508B6FF6D
:10205C000106C6A426F620D5047002D22B80D92402
:10206C00CFB41A00EF5004C2E5D22C0221E8D229D9
:10207C0080C6D22880C0D22A80BCD2D580BAD22DBC
:10208C0080B47F20121FD7202A077401B54100406D
:10209C00F1121F9CFF121FD7022010D230D22E80BB
:1020AC0095121F9CFB121F9CFA121F9CF94A4B7035
:1020BC000679B97A227BFF202A2EE541602A7E0020
:1020CC008E8275830012231160060EEE654270F04D
:1020DC00C2D5EBC0E0EAC0E0E9C0E0EE12222FD09E
:1020EC00E0F9D0E0FAD0E0FB1222F8FF60AAEBC0D6
:1020FC00E0EAC0E0E9C0E0121FD7D0E02401F9D03B
:10210C00E03400FAD0E0FBE5420460DCD542D98033
:10211C00877BFF7A22792BD22A809C7910800279D6
:10212C0008C22EC2308008D2D5790A8004790AC23E
:10213C00D5E542047002F542E4FAFDFEFF121F9C45
:10214C00FC7B08202913121F9CFD7B1030280A12DF
:10215C001F9CFE121F9CFF7B20EC3382D592D55026
:10216C0013C3E43028069FFFE49EFEE42029039D60
:10217C00FDE49CFCE4CBF8C229EC700CCFCECDCCAA
:10218C00E824F8F870F38017C3EF33FFEE33FEED5D
:10219C0033FDEC33FCEB33FB994002FB0FD8E9EB3E
:1021AC00302905F8D0E0C448B229C0E00AEC4D4E05
:1021BC004F78207B0070C2EAB5420040BCC0E012F0
:1021CC002231D0F0D0E0202904C4C0E0C4B229C030
:1021DC00F0121FC0D0F0D5F0EB02201012257D209C
:1021EC00AD53212758207E4C207A42212B4F21338E
:0F21FC0044213349209343213955211D46211D8C
:10220B0045211D4722D95020822D20862E20A92B17
:10221B00208A2320A72022C22A204248000020A186
:10222B003F3F3F00790AA2D5202B14302D09B9105E
:10223B00020404B9080104A2D5202E025001042087
:10224B002A68922AB541005034C0E07F20302B1908
:10225B007F30A22A722E722D500F122288C22AC2F0
:10226B002EC22DC2307F30800F302D03E9C0E0121B
:10227B001FD7302D03D0E0F9D0E0B541CC302D176E
:10228B007F30B9100C121FD77F58302C077F788006
:10229B0003B90803121FD7302A057F2D021FD77FE2
:1022AB00202030F87F2B202EF322922A80CF286E0D
:1022BB00756C6C2900D229121F9C3029F8C2297821
:1022CB004130D50108F60220422D50434958121FC8
:1022DB009C2403B405004001E49022D493121FC840
:0D22EB00743A121FC8D22B7541040221273E
:104579008B318A3289338B378A388939AB310533A4
:10458900E533AA327002053214F91222F870ED747B
:10459900FF2533F53374FF3532F532AB340536E593
:1045A90036AA357002053514F91222F8FFAB310528
:1045B90033E533AA327002053214F9EF1223717010
:0845C900DAAB37AA38A9392248
:102BB3008B2C8A2D892EE4F538F537F536F535F566
:102BC30033F534E5304531452F6012EBC0E0EAC000
:102BD300E0E9C0E0AB2FAA30A93112252EAB2C05BA
:102BE3002EE52EAA2D7002052D14F91222F8F539BF
:102BF300C394094007E539D3940D40E1E5396420D6
:102C030060DBE539B42D054334038016E539B42B75
:102C130005433401800C74FF252EF52E74FF352DEA
:102C2300F52DE53260046410703FAB2CAA2DA92E5C
:102C33001222F864306009E532702E75320A802959
:102C4300900001122311FF64786004EFB45813431A
:102C530034017532107402252EF52EE4352DF52D31
:102C63008007E5327003753208AB2C052EE52EAADA
:102C73002D7002052D14F91222F8F539C394614021
:102C83000AE539D3947A50035339DF74D02539F5E3
:102C930039C3940A400CE5399411406D74F9253910
:102CA300F539E539D39532506043340185383D8594
:102CB300373C85363B85353AAF327E00E4FCFDABCD
:102CC30038AA37A936A8351224CFC8ECC8C9EDC92C
:102CD300CAEECACBEFCBE4FCFDFEEB2539F538EEAB
:102CE3003AF537ED39F536EC38F535AF38AE37AD63
:102CF30036FCAB3DAA3CA93BA83AD312248150032E
:102D0300022C6C433404022C6CE53420E003E48091
:102D13002DE5304531452F601EAB2CE52E24FFF900
:102D2300E52D34FFFAEBC0E0EAC0E0E9C0E0AB2FE9
:102D3300AA30A93112252EE53430E20774FFFFFED5
:102D4300FDFC22E534AF38AE37AD36AC3530E103A8
:042D530002247322C1
:1024CF00E88FF0A4CC8BF0A42CFCE98EF0A42CFCAC
:1024DF008AF0EDA42CFCEA8EF0A4CDA8F08BF0A42A
:1024EF002DCC3825F0FDE98FF0A42CCD35F0FCEB89
:1024FF008EF0A4FEA9F0EB8FF0A4CFC5F02ECD394E
:0F250F00FEE43CFCEAA42DCE35F0FDE43CFC22BA
:10251E00FAE6FB0808E6F925F0F618E6CA3AF622BE
:10252E00BB011A89828A83D0F0D0E0F8D0E0F9D0CE
:10253E00E0FAD0E0FBE8C0E0C0F00225AC5016E9AE
:10254E00F8D083D082D0E0F9D0E0FAD0E0FBC082A0
:10255E00C0830225A3BBFE16E9F8D083D082D0E05B
:0F256E00F9D0E0FAD0E0FBC082C0830225B5228D
:10257D00D083D082F8E4937012740193700DA3A3ED
:10258D0093F8740193F5828883E473740293686001
:06259D00EFA3A3A380DF01
:0925A300EBF608EAF608E9F6225D
:0925AC00EBF0A3EAF0A3E9F02230
:0925B500EBF208EAF208E9F22257
:00000001FF
